:10000000C023002001010000FD000000FD000000F1
:1000100000000000000000000000000000000000E0
:10002000000000000000000000000000FD000000D3
:100030000000000000000000FD000000FD000000C6
:10004000FD000000FD000000FD000000FD000000BC
:10005000FD000000FD000000FD0000003510000064
:10006000FD000000FD000000FD000000FD0000009C
:10007000FD0000000000000000000000FD00000086
:10008000FD000000FD000000FD000000FD0000007C
:10009000FD0000000000000000000000FD00000066
:1000A000FD000000FD000000FD000000FD0000005C
:1000B0000000000010B5064C2378002B07D1054B3B
:1000C000002B02D0044800E000BF0123237010BDC4
:1000D000680000200000000038240000044B10B528
:1000E000002B03D00349044800E000BF10BDC04608
:1000F000000000006C00002038240000FEE7000033
:100100002549264870B581420AD0254BC41E0022DD
:10011000A34203D303331A1A92089200214B984743
:100120002148224BC11E0022994203D803331A1AD8
:100130009208920000211E4B9847FF221D4B03217D
:1001400093431D4A0C2593600222082430261B4B42
:100150001B485A62C3788B431343C370C378AB43C5
:100160002343C370174B987BB043060020203043D5
:100170009873987BA84304439C73987B88430243FD
:100180009A738023104A51680B4353600F4B984772
:100190000F4B9847FEE7C0463824000000000020BF
:1001A000680000205523000068000020BC030020E8
:1001B000672300000000000000ED00E0FC7000413B
:1001C0000050004100480041004000410D23000064
:1001D000611A0000F0B517000A7885B053060C00CC
:1001E00001909B0F012B52D1637909792A4D1B0293
:1001F0000B432978994202D06978994247D1E67930
:10020000A379360252B21E43002A0FDA0020012FD2
:100210000AD06378212B11D1072E3BD10300A91DF1
:10022000320001981D4CA04705B0F0BD1C4B98470B
:1002300063780100202B03D0222B19D00D2027E05A
:10024000072E27D1002F01D13B00E9E73200154CE2
:1002500002A8A0472B69002B05D10722A81D02A9DF
:10026000A0470020E0E702A898470028F5D1F8E76A
:1002700000230A4E1A0019001800B0476B69002BC2
:10028000EFD0E078A278000210439847E9E70A200F
:100290004042C9E70120FBE784000020811E0000E6
:1002A000A922000055230000F7B5150001294FD001
:1002B000022900D176E0002900D075E0836810683B
:1002C0001E00009302330193002802D10A2040420D
:1002D00020E00821437982788B43022BF6D13378D2
:1002E0009A4263D0FF2B63D1327069680522324B8A
:1002F0009847041E0FD12868042203786968C01843
:100300002D4B9847019B0136B342DDD101222000DD
:100310002A4B5A71FEBD637922791B02A778D21845
:100320003800E178264B92B29847002842D17BB240
:10033000244A002B09DAB770380090472C602078E7
:100340006968214B20189847D3E7009B1F71F3E79A
:100350008468002A05D0136808225B799343022B36
:10036000B4D12378FF2B07D0FF25A0782570A842B1
:1003700002D0164B9847A5706378FF2B07D0FF2556
:10038000E0786570A84202D0104B9847E57020795C
:10039000FF2803D00D4B9847FF2323710020074B04
:1003A0005871B7E71B2092E70D2090E712208EE7E7
:1003B0001C208CE714208AE7E5140000840000204C
:1003C000F117000081180000FF140000551800000C
:1003D00010B50A4B984701280CD80948094B006210
:1003E000C361094B1830984701200849084B9847CA
:1003F000002010BD11204042FBE7C046B52200009E
:1004000084000020A902000051220000000000200A
:10041000C521000000207047074B9A8C920604D536
:100420001022D9681142FCD004E0D021DA680A40D9
:10043000D02AFBD17047C04600080040002803D0F6
:10044000002901D00230C0B2142301305843014BBF
:10045000C0187047080100200F2370B50100807C90
:10046000072503401A00CC7C083225405B01012D92
:1004700008D01449520152181021D171124A9B1808
:10048000597270BD40252C4206D08026AC43CC74F6
:100490000D4C1C196671A5710825CC7C5201AC432A
:1004A000CC7400240949C9188C728C7605495218FD
:1004B0006F21D171044A9B185972054B9B6898476C
:1004C000DFE7C04600500041FF500041A800002077
:1004D0000801002020238B40DAB20F2310B504005E
:1004E000807C054903405B015B185A72034B012174
:1004F0001B69A268984710BDFF5000410801002009
:1005000010B50300807CFF2809D04024DA7C224209
:1005100005D0A243DA74024A14699A68A04710BD54
:1005200008010020F7B59446837C134A01AE0D0004
:100530003280FF2B1AD04027C27C3A4216D00F22BD
:1005400013401C0008346201002910D00B4FD2194F
:10055000802717710949640164180949725D5B01BC
:100560005B18E27161465A72064B9847F7BD034922
:1005700052185771EEE7C046254A0000005000416E
:10058000FF50004101050000F0B50D000F21837CF4
:1005900085B00B409C46304B03AE338063465B0115
:1005A0000093634608332D495C01002D20D0095D7E
:1005B0004906490F009A2C01A418294A765D14199E
:1005C000A77AFFB2022917D101390F4214D0A77AB6
:1005D000224A5B019B188F43009AA772DE71214B60
:1005E0002940D218567204221F4B984705B0F0BD1F
:1005F0000C5D07212140DDE702213A000A4001920B
:100600000F4217D0A27AC77C8A43A272134A5B01B9
:100610009B18DE71009A134BD218072356723B4089
:10062000012BE3D17B06E1D5C17CC909A942DDD00C
:100630000022D9E7624651004D19094A2D0155198A
:10064000019A5B01AA72054A9B18DE71009A054B5C
:10065000D2185672CAE7C046040800000050004194
:10066000A8000020FF5000412505000070B5FF26BE
:10067000084D094CC83503212000084B984700213C
:10068000A674E1741434AC42F5D16022044B0548E1
:10069000984770BD080100201C01002001050000E2
:1006A00067230000A8000020F0B50F2785B0019156
:1006B000837C040002931F400023994205D04B4BDA
:1006C0007A019B185B699B049B0C258A484AAC46BF
:1006D000954202D06A1E12B294460722E07C024084
:1006E0000392019A002A04D042497A015218022149
:1006F000D171A26899186268A160914240D22368C2
:10070000521A59187B01394E92B2029383062CD5A6
:100710002B1C954200D9131C9DB22A00364BE06871
:100720009847324BE26879015B181A617B01F61831
:100730007369AD049B0BAA0C9D0315437561736926
:100740002E4A13407361019B002B08D1039B4E225C
:10075000012B00D0043A2A497B015B189A72254A82
:100760007B019B1880225A7139E08023151C9B0164
:100770009A4200D91D1C7B01F318ADB21961D5E76F
:1007800010267A0130420ED0E37C1C49B343E37457
:10079000164B9A18921953689B0B9B03536053682E
:1007A0000B405360CFE7039801281AD11448121860
:1007B0004B205072624613409D420CD14025E37C91
:1007C0000298AB43E3740F4BDB689847002806D1CF
:1007D000E37C2B43E374002120000B4B984705B0CA
:1007E000F0BD074812184A20E3E7C046A8000020E1
:1007F000FF0300000051004155230000FF3F00F0BF
:10080000FF50004108010020010500000F23F0B552
:10081000857C85B004000E001D40039101910029E4
:100820000AD0614B6A019B18596809018A0C03922E
:10083000596889048B0C0193238A0093009A5B4BBF
:100840009A4203D01300013B9BB20093019B009F8F
:10085000E27C1F40072313400293002E04D054492A
:100860006B015B180121D97193060FD56368002BCA
:100870000CD0A26821689B1A88181A1C9BB2BB4234
:1008800000D93A1CE1684B4B92B2984763686A0101
:100890009446002B2CD1E27CD10629D530339A43E3
:1008A000103B1A43E2746246E1683F4B424899505C
:1008B000218A63445A688904090902400A435A603C
:1008C0005A68920B92035A60002E0BD1029925228E
:1008D0006B01012903D1344AD21896762D2237496B
:1008E0005B189A72324B6D01ED1840232B711DE09D
:1008F000A168002E1CD0228ABA4219D91022E37CAA
:100900009343E374019B5918A160029A6B01012A79
:1009100046D12A4A9B182D225A72002D02D1224B11
:10092000E2681A6000212000254B984705B0F0BD11
:10093000039A5118A1608B42E7D92020E27C5B1A10
:10094000278A9BB2024216D0391C9F4200D9191C3B
:10095000E068154A8BB269015050134A1648624448
:1009600051689B041B0901400B43536053689B0B68
:100970009B035360A8E79F420BD2802080018342F3
:100980000CD8009A93432068074A41186801115017
:10099000E3E79F42F7D91043E074F4E70300F2E77E
:1009A000064A9B182522B7E7A8000020FF03000095
:1009B0000051004155230000FF3F00F0FF5000416F
:1009C00001050000802302009B0007209A4214D8F2
:1009D000013BFF3B01389A420FD80138802A0CD8DE
:1009E0000138402A09D80138202A06D80138102AAF
:1009F00003D80630904280414042704710B52A4CDF
:100A0000A378DB0718D40323A2781A42FCD1022270
:100A1000237813420AD02378934323700323A278C8
:100A20001A42FCD10223A2781A42FCD1012323707E
:100A30000233A2781A42FCD10123A2781A42FCD1D7
:100A40001A4B1B4A1A605A609A60DA601A61194B95
:100A500098471F20184B1A68530B910C92010340C2
:100A60000140520F834200D105231F2900D10239D2
:100A7000072A00D1023A9B010B431203134323853B
:100A80000323E2781A43E2700C22E1780A43E27011
:100A900004222270A278100018401A42FAD1074BA3
:100AA00063620123238110BD005000410801002032
:100AB000150400006D06000024608000A8000020DE
:100AC00003220E4B9978114214D199781142FCD12E
:100AD00002221978C8B2114205D102431A700322CA
:100AE00099781142FCD180210020054A1160054A05
:100AF0001A83704711204042FBE7C0460050004176
:100B000000E100E08D0200000121024A13898B43BD
:100B1000138170470050004180231843014B9872A5
:100B20007047C04600500041F7B50F2404402E4BDB
:100B300000910600C10947B22000019298470321A5
:100B4000009B05000B400093022C44D8837CFF2BB4
:100B500044D1009B002B10D1F943C9B2224B200095
:100B6000C9099847837CFF2B38D1F33B63431F4A65
:100B70009B58002B34D113202EE0002F14DA0C22C6
:100B800062431A4B9B185A68002A19D10C236343FD
:100B9000164CE418636800200099EB60019B01315A
:100BA0002B82E974AE74FEBD0C2363430F4A9B583D
:100BB000002B0BD00C2262430C4B9B181B8900E0CE
:100BC0005B89019A9A42D6DC002FDFDB0C235C4361
:100BD000064BE358DFE712204042E4E71420FBE72E
:100BE000002FE7DACBE7C0463D0400007823000081
:100BF000F7B50F2504000540022D1AD843B2C709E6
:100C000001933900144B28009847837C0600FF2B82
:100C10000FD00322114B390098470722F37C134071
:100C2000012B07D100220E4B08346401E254FF234C
:100C30007382F7BD63B2002B07DA7022094B6D0196
:100C4000ED186B7893436B70F1E7064B6401E41881
:100C5000637893436370EAE73D04000025050000D4
:100C600000500041FF500041F7B50F240440C10976
:100C7000474B45B220009847464B6101CE18727829
:100C80000700D2B2022C00D97DE0837C0193FF2BB8
:100C900000D178E0404B5C18C37C07211800084065
:100CA00001283BD177231100194000911A4200D04E
:100CB0006CE0663B73703D8A384B28009847E02310
:100CC000374ADB0500071840AB031340034363605A
:100CD000402180230F22AD04AD0C28436061B17127
:100CE0007371009B2C48A372A376019BAC03134045
:100CF000FA685B011A50C01842682A4D1540254316
:100D000045604268920B92034260224A00989B1809
:100D1000B0225A71A03A99719A72FEBD002D19DA6B
:100D2000702115000D400A4230D15B075B0E134362
:100D300073703F8A194B38009847E0230007DB05A2
:100D400018408023BF04BF0C384360617371A576DF
:100D50002800E2E715000D400A4217D15B075B0F40
:100D6000134373703F8A0D4B380098470C4ABB03FE
:100D70001340E0220007D205104003436360402384
:100D8000B371A572E4E712204042C6E71420FBE7E6
:100D90003D040000FF500041A8000020C5090000EC
:100DA00000C0FF0FFF3F00F0F8B507000F26C40991
:100DB00037400D0038002100294B98470200022FD0
:100DC0004AD8837C10203340A040012D10D1254DFE
:100DD0005901C0B2491948712021A14022485B0144
:100DE000C9B21B1899720823D17C0B43D37409E054
:100DF0005B01002D29D11D495D181B495B18D9796C
:100E0000084201D100201CE02021A140C0B258714D
:100E1000C8B258721E7A314204D00121A140C9B231
:100E2000187259710721D37C194001290AD1FF3565
:100E3000EC792F31200008400C42E3D128398B4354
:100E4000D374F8BD08218B43D0E7064A9B189B79E1
:100E50001840431E9841F4E712204042F1E7C04693
:100E60003D04000000510041FF500041005000418E
:100E7000F8B50F231840114B44011B190F001968D6
:100E80005D68AD04AD0C022812D8002F10D00C4BB9
:100E9000E4186378112B0ED11026227A00203242FA
:100EA00005D008223800074B984728002672F8BD65
:100EB00012204042FBE71320FBE7C046A8000020B9
:100EC000FF50004155230000F0B50F25077A87B089
:100ED0007BB23D40FF093900029306003A4B2800DF
:100EE00098473A49038A04001A008B4201D05A1EDF
:100EF00092B271680A400192022D62D88020326855
:100F0000800582420DD3324D8818A84209D80320AB
:100F100015000540024204D1029A002A0EDB9942D4
:100F200006D2E3680125002B08D11320404217E0C8
:100F3000019B002B16D0E368002B42D0E37C0220FB
:100F40001B070DD4234B05A89847E17C40230A00DA
:100F50001A400392204A194206D005A89047012062
:100F600007B0F0BD019DE9E70B43E37405A8904786
:100F70007F213368FA0123607368039F6360039BDA
:100F8000A360E37C0B40134369011D0020239D43B4
:100F90000D43E574737A002B02D0019F7B425F41C1
:100FA0001022E37C3F0193431F43029B002120005A
:100FB000E774002B03DA094B98470020D0E7084B71
:100FC000FAE71220B2E7C0463D040000FF0300002C
:100FD000FF7F0020C9220000D7220000A9060000E0
:100FE0000D080000002900D10549012802D1054B58
:100FF000596070470028FCD1024B1960F9E7C046E0
:101000001504000008010020002900D1074900282C
:1010100002D1074B99607047012802D1044BD96077
:10102000F9E70228F7D1024B1961F4E71504000033
:1010300008010020F7B56C4B1A8C91B20191002A7F
:1010400000D066E09A8B198B04200A401100014001
:10105000024204D09883654B1B689847F7BD8024F3
:101060001600A400264022421DD0614A9A839A822B
:10107000923AFF3A1A835F4B1A891207120F032A1A
:1010800005D01A8D1207120F032A07D10121002261
:1010900049015B1819891A814904490D0320534BF2
:1010A0005B689847DAE7802415002540224205D086
:1010B0009C834E4B310005205B68F2E770261400DC
:1010C000344032420AD04A4A9E839E821A834A4B57
:1010D0009847464B290002205B68E2E7082511008B
:1010E00029402A420CD0454A5470414A9D839E8231
:1010F0001A83434B98473D4B210001205B68D0E7A2
:10110000D20706D53A4A9A839A821E83374B5B6888
:10111000C7E700260F2701253A4CA37CFF2B38D0C8
:101120002A003B409A400199114232D036495A0177
:10113000521832495B015B181278997A0B00134000
:10114000114226D014217143284A521847211032E7
:10115000D27D1140012911D1DA0603D520002B4B95
:10116000984716E0402219001140134201D029008F
:1011700001E09B060DD52000254B09E051B2002966
:101180001CDA5906F3D4190708D529002000214B91
:10119000984701361434092EBFD15FE7990703D56C
:1011A000290020001C4BF3E707210A40012AF0D157
:1011B00000215A07EAD4DB06EBD5CFE7202019003F
:1011C0000140034201D00021D5E75807DED42B426D
:1011D00003D029002000114BDAE707210A40012A39
:1011E000D7D11A07E7D5D0E7005000410801002009
:1011F00001020000A800002019040000FF50004177
:101200006D0600001C010020075100415904000038
:10121000D504000089050000A90600000D080000A3
:10122000064B1A7AD2B21A725A7AD2B25A729A7A91
:10123000D2B29A72DA7AD2B2DA72704700040040FF
:101240000423074A10B551680B435360054B984778
:10125000054B9847054B9847FF20054B984710BD15
:1012600000400041211200000D1300003513000062
:10127000A91400000068002800D170478842F9D105
:101280000120FAE770B50C4B05000C000668984782
:10129000012358404F22094B0949C0B298472B6897
:1012A000002B02D12C60236070BD33003668002E05
:1012B000FBD11C602660F7E775120000C512000024
:1012C0009C230000002800D100BE7047064810B5DE
:1012D000064B40309847064B9847064B06489847C0
:1012E000064B984710BDC04690020020F121000037
:1012F000D103000069220000080000209D220000A8
:1013000010B5014B984710BDCD1200000E22084BBE
:101310009A8299690C3A0A431F219A611A7F0A40FE
:101320001A771E39DA6852080A42FBD07047C04665
:101330000008004002220121144B9A84DA68120945
:101340000A42FBD0124ADA62FC22D2019A62972248
:1013500052009A849A8C92080A4210D01022D968BE
:101360001142FCD08022998C0A430A499A844A7817
:10137000D209FCD102219A698A439A6170470121FE
:10138000DA6812090A42FBD0ECE7C04600080040C8
:1013900080BB0104000C0040F8B506000D001400ED
:1013A000002804D0081E02D01000431E9841F122EC
:1013B0001049114B98473700083738000F4B9847B2
:1013C0000028F8D000263800A95D0D4B984738005A
:1013D0000A4B98470028FAD00136B442F3D80125C9
:1013E000002C00D025003800064B98470028FAD082
:1013F0002800F8BDBA230000C5120000CB1C000075
:10140000BD1C0000D51C0000F7B5050014000191BB
:10141000002804D0081E02D01000431E98418622E6
:101420000C490D4B5200984700262F000837380012
:101430000A4B98470028F8D0094B38009847019B81
:1014400098550136B442F0D80120002C00D020007D
:10145000FEBDC046BA230000C5120000DF1C00001C
:10146000C31C000070B504000D00002802D0080065
:10147000431E98410749084B342298472000290011
:10148000064B08309847002803D1054B6360054B95
:10149000236070BDBA230000C5120000911C00003B
:1014A0000914000099130000C30708D580230A4AD5
:1014B0005B009360094B53605378DB09FCD18307D1
:1014C00008D50223044AFF339360054B53605378D9
:1014D000DB09FCD17047C046000C0040000701004A
:1014E0000105010010B5884201D3002010BD03782A
:1014F000012BFAD944789442F8D0C018F3E7884217
:1015000001D3002070470378012BFAD94278042ACE
:10151000F7D0052AF6D0C018F1E7000070B50D4BE2
:10152000150002220C00984700280FD170BD0378E7
:10153000012B0DD94378022B0AD14379AB42F5D068
:10154000C278837812029B189BB2C018A042EED3D7
:101550000020EBE7E514000070B50C001600002534
:10156000A04201D3002070BD03222100054B984703
:101570000028F8D00378012BF4D9B542F3D0C01875
:101580000135EDE7E514000002000F21002030B521
:10159000094B11405C7894420CD01D78002D01D18C
:1015A0008C4207D00130C4B2203340B2042CF1D1B8
:1015B0000120404230BDC04610030020002070478B
:1015C00070B5084B04000D009847074B40011B18ED
:1015D0009A780020032A03D1290020009B699847AC
:1015E00070BDC0468915000010030020F0B5374BD0
:1015F00087B00F00009001929847354D4401002FAD
:1016000041D12E19F770295D002933D12200B47819
:101610000C327078F369AA18032C27D10C270131FA
:10162000F757984703007078002B0BD0294B738035
:10163000002F02DB863BFF3B18430121264B9847D6
:1016400007B0F0BD04220393B2700493002F0ADBAD
:101650008023184302AB1873012302AA537303A813
:101660001E4B9847ECE70F231840F3E798470223F7
:10167000B370E5E70123B3702C19E178E369019AAF
:1016800000989847DCE72B19012F0CD10222DA7061
:10169000295D002904D19A7000980F4B9847EBE719
:1016A00005229A70E8E7022F08D10422DA702A5D39
:1016B000002A01D19F70C3E70122F2E7032F03D173
:1016C000A022D2005A80D7E7054AFBE7891500001F
:1016D0001003002005020000A90D0000C90E000043
:1016E00006060000F7B5184B0400984747013B0079
:1016F000164D0C335B19190001932000144B9847C9
:101700008026C0B226430096124E082806D001213A
:101710002000B04701210098B047F7BDED1901271F
:1017200000212000B04700210098B0472000019917
:101730006B69AF7098470028EFD10523390020006E
:10174000AB70B0473900E6E78915000010030020B0
:10175000710E0000A90D000070B5114B98470028CC
:101760001DDB104C8022002120000F4B98472300E6
:10177000FF2104240D4A013CE4B259705A619A6178
:10178000DA612033002CF6D1094D20000949A84721
:1017900001200949A84702200849A847200070BD38
:1017A000FD0900001003002067230000BD150000A4
:1017B00009100000E5160000C1150000ED1500003D
:1017C00010B5014B984710BDE50F000010B5014B57
:1017D000984710BDC10A000010B5014B984710BDD5
:1017E000090B000010B5014B984710BD190B000004
:1017F000F8B5104C06000D001700A047002813DABA
:10180000FF20A047041E12DB3A00290030000A4BDB
:101810009847002807DB03210020084B64011A19B0
:101820000D405670E554F8BD14204042FBE71520EA
:10183000FBE7C04689150000290B000010030020BB
:10184000002110B502000800014B984710BDC046AA
:10185000F117000070B5074B05009847041E07DB21
:101860002800054B9847FF2304486401041963705E
:1018700070BDC04689150000F10B00001003002068
:1018800070B50C4B0400984700280FDB0A4D40014F
:10189000425D2D1851424A4101322000074BAA7087
:1018A0009847002801DA0023AB7070BD1220404237
:1018B000FBE7C0468915000010030020690C0000FA
:1018C000F0B5037A04008BB018000193324B9847AF
:1018D000637A061E656802935BDB304B06A8984767
:1018E00073010093009A2E4B9E18B37804AAD71D5B
:1018F0003B703A78D3B203932A4B012A1DD10232AE
:10190000B27006A89847264B009AD35C002B1FD0D4
:101910000298019B421E9041D909C0B22368227AE5
:1019200007930895002931D080231A4304AB1A7518
:1019300058751D4B07A8984708E006A898473B78BC
:101940000120DAB2062B01D8184B98560BB0F0BD27
:10195000F27CB37C12029B189BB2002B05D10422AF
:1019600003981D000100B270D8E79D4200D91D0008
:101970000B4900208C46009A01006244127B7F2AAA
:10198000CCD99D429B4101315842C7E70F231A40F1
:10199000CCE712204042D9E789150000C922000097
:1019A00010030020D7220000C90E0000D62300003B
:1019B000F8B505000E1E1AD1124B9847041E1DDB08
:1019C00002212800104FB84700280FD0310028000E
:1019D000B84700280ADB0D480D4B640124186380CA
:1019E000320003212800E36998473000F8BD064B18
:1019F000012900D0022128009847F7E71220404231
:101A0000F4E7C04689150000A90D0000100300206E
:101A10000103000070B50F4B14000D009847002C17
:101A200000D10D4C002809DB012D08D0022D0BD070
:101A3000002D03D1094B40011818446170BD074BBC
:101A4000400118188461F9E7044B40011818C4617B
:101A5000F4E7C04689150000BD1500001003002002
:101A600010B5014B9847FEE7E91C000030B5012492
:101A70000C4BC5B2C0180378CAB2A3430A4923432A
:101A800003706B085B180F201978254205D00140C0
:101A900012011143C9B2197030BD81430A431A7053
:101AA000FAE7C046404400413044004110B51620DA
:101AB000034C0449A04717200349A04710BDC04666
:101AC0006D1A000002001600020017002023044ACD
:101AD000116A0B431362034B034A5A807047C04696
:101AE00000040040000C00401740000010B5054BFA
:101AF000984700220449054B05489847054B9847ED
:101B000010BDC046CD1A000000140042651400004C
:101B100090030020AD1A0000F8B5C025802380276F
:101B2000114C124AED05FF055B04AB60A762A2628F
:101B3000220004266B61583213781820B3431370C7
:101B40000B490C4B984780230B4A9B04AB60A76260
:101B5000A2626B61593423781920B343237007497B
:101B6000044B9847F8BDC04600440041000100C046
:101B7000060018006D1A0000000200C006001900DF
:101B80002022064BD9690A43DA61402259690A4387
:101B90005A61034B034A5A807047C0460004004014
:101BA000000C00400640000010B5034B9847034B63
:101BB0009847034B984710BD811B00005917000040
:101BC000191B000010B5034B9847034B9847034B74
:101BD000984710BD41120000ED1A0000A91B00003B
:101BE000C3691942FCD17047022210B50368032172
:101BF00093430360014B984710BDC046E11B0000B2
:101C00001B4B70B5C3189B0ADBB20400032B04D036
:101C10000020184A1849194B9847E369184DDB070B
:101C200011D4022603212000A8472368334205D09F
:101C30002000144B984731002000A84705230321BA
:101C400020002360A84720000121A8470E4B200058
:101C500023600321A847C0239B0220006360072163
:101C6000A8470020094BA381A0733034207070BDB9
:101C700000F8FFBD3A020000E4230000C512000096
:101C8000E11B0000E91B0000040010402BF6FFFFE1
:101C900070B50500431E98410C00B4220449054B61
:101CA000C0B298472C602000034B984770BDC046D7
:101CB000E4230000C5120000011C00000368198520
:101CC00070470368188DC0B270470368187E0123FF
:101CD000184070470368187E8007C00F704703687C
:101CE000187E4007C00F704710B5024B9847024B53
:101CF000984710BDC51B000001130000064B10B52E
:101D00001C69002C00D110BD200063680022012155
:101D100098472468F5E7C0469C03002070B505008D
:101D20000E00064BDC68002C00D170BD6368002BF0
:101D300002D03100280098472468F4E79C03002073
:101D4000F8B505000E0017000B4B9C68002C01D164
:101D50002000F8BD6368002B01D12468F6E73A0043
:101D6000310028009847002804D00A30F5D001201F
:101D70004042EEE70120ECE79C030020054B10B544
:101D80005C68002C00D110BD6368002B00D0984720
:101D90002468F6E79C03002010B51400002903D046
:101DA000012923D0002010BD1378002BFAD15378DD
:101DB000052B0FD0092BF5D1E17892780E4B090253
:101DC0001143D9764A1E91410331997601200B4B7C
:101DD0009847E7E70A4B90789847E178A27809029C
:101DE00011434B1E9941044B0231EEE70A00054BAB
:101DF000210000209847D5E79C0300201D1D00000E
:101E0000E5170000411D000070B5002402260C4BB0
:101E100098470C4D20006E830B4B6C7798470B4B0B
:101E2000287F98470A4D210020000A4AA847310020
:101E30002000094AA8472000084B984770BDC046BB
:101E4000FD1C00009C0300205518000041180000F4
:101E5000151A00009D1E0000991D00008118000049
:101E600010B5002802D0012803D010BD024B9847BE
:101E7000FBE7024B9847F8E71D1D0000091E000014
:101E80001FB502926A461073537301A8024B019169
:101E9000984705B000BDC046C1180000F7B5B74B64
:101EA000002204000D009847030000205A1C00D1B6
:101EB000C1E00130834200D1BDE02B781F22190020
:101EC000914304D0802900D1B6E00020B3E06878C7
:101ED00001380A28F9D800F005FA46F856F80BF848
:101EE000F8F806F86000AA78002A0BD1A44B9847AE
:101EF0000022012311002000A24CA0474342584178
:101F0000C0B298E0A04D2B6803CBA04B98470028A7
:101F100000D190E0C37881781B02C91889B24118BA
:101F200004229B4B01919847FF220090009B002BBD
:101F3000DED09E78964202D02F69002F0AD10098F9
:101F4000042203780199C0180090914B9847320001
:101F50000090EBE76A46002138007B68984700282C
:101F6000EDD03F68E9E7022BAFD1EE79AB793602CD
:101F70001E43AAD131002879864B984701233200AD
:101F80003100200054E0022B9FD1EB79AE791B0287
:101F90001E439AD101212879EEE7EC78AB78240230
:101FA0001C432B796D79784E2D021D433368F27EE8
:101FB00003CB764B9847002887D004220090C37843
:101FC00081781B02C91889B24118714F0191B84735
:101FD000002800D179E78378AB4210D1C378A342BF
:101FE0000DD137690090002F00D16EE701216A46BC
:101FF00038007B689847011E08D03F68F3E70098D7
:10200000042203780199C0180090E0E76A4638007E
:102010007B689847002800D057E7002C04D00122A5
:10202000AA40737F1343737700231A001900180026
:10203000544CA0470120FEBD68780A2800D944E727
:1020400000F05AF9620043FF43FF43FF43FF43FFA1
:102050000B0043FF5A0043FF8300E978AB78090285
:102060000B43090ACAB2022917D0032A34D0002030
:10207000012AE0D1AB79ED792D021D43424B1B685B
:1020800003CB434B9847011E00D11EE72A1C122D9B
:1020900000D91222002392B22DE7AA79ED790133FB
:1020A0002D021543384A1068167F03C8DAB2374B41
:1020B0009847011E00D108E7C37882781B02D21826
:1020C00092B20023954205D9013E35406B425D41F5
:1020D000EBB215002A000EE7AA79ED792D0215431F
:1020E000294A1068167F03C8DAB22B4B9847011EA5
:1020F00000D1EAE60278E4E72349CB7E4A6913700F
:102100004969002301223CE71F211E2218001940C3
:10211000104013420ED0022900D0D6E61D4B28797C
:10212000984703000020834200DA84E7013003402F
:10213000009300E00090144D02226946174B686935
:1021400098470023022269691BE70F4E6B792979B2
:10215000727F1B020B431A410124100020402242CF
:102160001ED03469002C00D1AFE62A0002212000E5
:102170006368984700281BDA2468F3E7411D0000D4
:10218000FD1C0000811E00009C0300201D150000A6
:10219000E5140000B1190000591500005523000096
:1021A00073692200187071690300054DA84741E763
:1021B00073690122187000237169180038E7C0465E
:1021C000811E000010B5012808D0022809D000287F
:1021D00003D105480430054B984710BD024808302C
:1021E000F9E701480C30F6E79C0300208512000057
:1021F00070B50400431E98410C4A0D4B0D49C0B206
:1022000098470D4B984700280EDB0C4D20220C4BB5
:1022100000212800984700200A496C610A4CA04719
:1022200001200A49A047002070BDC04655030000A8
:10223000C5120000FF230000591700009C03002076
:10224000672300007D1D0000C1170000611E000013
:1022500010B501000248034B1030984710BDC0462E
:102260009C0300208512000010B50A4B9C7E002CB8
:102270000BD100280CD002681860D2791A7701229D
:102280009A76054B9847200010BD04204042FBE79A
:102290000920FBE79C030020CD17000010B5014B7F
:1022A000984710BDD9170000014B58697047C046C8
:1022B0009C030020034B987E1023184200D0180086
:1022C0007047C0469C030020EFF31083036072B692
:1022D000BFF35F8F7047BFF35F8F036883F310888E
:1022E0007047000002B47146490849000956490088
:1022F0008E4402BC7047C04603B471464908400092
:102300004900095E49008E4403BC704770B5002641
:102310000C4D0D4C641BA410A64209D1002600F000
:102320007BF80A4D0A4C641BA410A64205D170BD6F
:10233000B300EB5898470136EEE7B300EB589847E7
:102340000136F2E7242400002424000024240000A5
:1023500028240000002310B59A4200D110BDCC5CA7
:10236000C4540133F8E703008218934200D1704748
:1023700019700133F9E7000050020020000000004E
:10238000400000001002002000000000400000009B
:10239000D001002000000000400000002E2E2F6819
:1023A000616C2F7574696C732F7372632F75746908
:1023B0006C735F6C6973742E63002E2E2F68616CD2
:1023C0002F7372632F68616C5F75736172745F73D2
:1023D000796E632E6300ED0101010102F0ED000151
:1023E000010102F02E2E2F68706C2F736572636FDF
:1023F0006D2F68706C5F736572636F6D2E63002E56
:102400002E2F7573622F6465766963652F7573620D
:1024100064632E6300000000F8B5C046F8BC08BC39
:102420009E467047DD000000F8B5C046F8BC08BC09
:082430009E467047B500000054
:1024380000000000D5010000100000206500002009
:102448001201100202000040EB0304240001010203
:10245800000109024300020100A032090400000142
:1024680002020000052400011005240101000424D3
:10247800020205240600010705820340000A090438
:102488000100020A000000070501024000000705DC
:08249800810240000000000079
:00000001FF
